:10000000902AA0007F39201B803C0920A01B003CC7
:1000100008008A01820700340334063409340C34A2
:1000200010341334163419341C341F34223425345C
:1000300028342B342E3431343334363439343C3490
:100040003F3441344434473449344C344E345134D1
:100050005334553458345A345C345E34603462342A
:100060006434663468346A346B346D346F3470349D
:1000700071347334743475347634783479347A3432
:100080007A347B347C347D347D347E347E347E34EB
:100090007F347F347F347F34A800F839A000A00C6F
:1000A000A00C200C8407D421A80000050800280813
:1000B000031C03010006280580068B2ACF21B80007
:1000C0000408BA000800CF21B9000408BB000800EA
:1000D000A4002508A402031CA5032708A602031CEC
:1000E000A7032508A00024080310A40DA50DA40D46
:1000F000A50DA4070318A50A2008A5072708A00036
:1001000026080310A60DA70DA60DA70DA607031818
:10011000A70A2008A7073B09A2003909A300A20AE1
:100120000319A30A0D30A900AC01AD01AE01AF0166
:10013000A8013A0884003808CB2184138C222408B3
:10014000AC070318AD0A2508AD072608AE0703184B
:10015000AF0A2708AF072D080120803EA1002F0815
:100160000120803EA107210CA80700083804031CC9
:1001700038068000290303190D30A9000319A20ACB
:100180000319A30F9E288B2A003803198B2AA80075
:100190002008840021188317A001A101A81BD828DA
:1001A0000008A000840AA81C8B2A0008A1008B2A42
:1001B000D4210005031DA00A8B2A2C08A0002D08BD
:1001C000A1000130A20064000521031CF228A20B4B
:1001D000E328FF30A007031CA107031C8B2A323041
:1001E000A200E3288D21A8010830A3008E2105215B
:1001F0000318A80AAB1EA801A20CA30BF628AB1A81
:10020000A2138E210314220808003A08840038083B
:1002100084178004841300052B1B3806FF3E08005A
:10022000A401A501B7128622031C0800D33E0319BE
:10023000B7162D3EC63E031813290A3E031C132988
:10024000A2000310240DA000250DA100200DA10D7A
:10025000A4070318A10A2108A507A40DA50D2208CB
:10026000A4070318A50AA90303193F298622031C22
:100270000800C63E03183F290A3E03182029B71E6E
:100280004629A409A509A40A0319A50A24080314E8
:100290008B2AA600822103184A2950290408A600A7
:1002A0003A088400F030B7050830A700031003189F
:1002B000B70A6821A60CA70B57290000AB1A370C08
:1002C00068218E22031468212F08A3002E08F82924
:1002D0008413AB1F7729000838042B1F38068000D1
:1002E000841700083804031C380680008E29000893
:1002F0003804031C38062B1B380680008417380985
:1003000080058E293B0884003908841780048413F3
:1003100000052B1B3906FF3E080037172B081F3935
:10032000FF3EA1002A08F53E0318A10A371F052A3F
:100330003713A00002303222052AB7132908031907
:10034000B7170530A8002730A3001030B3210330C1
:10035000A300E830B321A3016430B321A3010A3024
:10036000B3212408BA29A2002508A1002408A0006E
:1003700054222008A000A8030319B7132908031961
:10038000C4292802031808002008031DB713B71B4F
:100390000800303E862AFF3A841780058B2AA80081
:1003A0000630A8190730840001308A002808073970
:1003B00082070134023404340834103420344034C9
:1003C000803403178D0083168C130C1483120C08D1
:1003D0008B2A03178C0083168C130C1555308D0057
:1003E000AA308D008C148C18F3290C118B2AA301D0
:1003F000A200FF30A207031CA307031C8B2A0330B3
:10040000A100DF300522F929A101E83EA000A109E1
:10041000FC30031C0E2AA00703180B2AA007640057
:10042000A10F0B2A2018142AA01C182A0000182A31
:100430000800A101A3013F221F2AA3013C220319A6
:10044000252A2308A1002208A00020080800031084
:10045000A00DA10DFF3E0318272A20088B2A0310A8
:10046000A10CA00CFF3E03182F2A20088B2AA10103
:10047000A301A2000230442AA2000130442AA200B3
:100480000430442AA2000530A80023082102031DDD
:100490004B2A2208200204300318013003190230CD
:1004A0002805031DFF308B2A1030A600A501A401EA
:1004B000210DA40DA50D2208A4022308031C230F5F
:1004C000A50203186A2A2208A40723080318230F89
:1004D000A5070310A00DA10DA60B582A20088B2AF2
:1004E0001030A800A101A001A70CA60C031C7E2AB5
:1004F0002208A00723080318230FA107A10CA00CB2
:10050000A50CA40CA80B742A24088B2A840031089B
:100510008A003008820083130313831264000800EA
:10052000831606309F0006309F0083125430BC00B3
:100530004030BD0064008A110A120518A52A8A11EC
:100540000A128C30BC004130BD005130E8000D3043
:10055000E121F0000E30E121E9000F30E121EA0055
:100560001030E121EE000515831605118312851068
:1005700083168510851005118312FF30C000FF30EF
:10058000C1000F30ED000730BA008030B8003C08E1
:10059000AA003D08AB00AE01AF0100304F21423050
:1005A0004F2175304F2167304F2120304F2143308C
:1005B0004F216F304F216D304F216D304F21613011
:1005C0004F216E304F2164304F2165304F21723002
:1005D0004F2120304F2142304F214F304F21533097
:1005E0004F2120304F21A9012A30A400A5014E300F
:1005F000B0000130B1009D212C304F2120304F211F
:100600004D304F2169304F216C304F2166304F21E2
:100610006F304F2172304F2164304F2120304F21F5
:1006200049304F216E304F2173304F2174304F21AC
:1006300072304F2175304F216D304F2165304F2181
:100640006E304F2174304F2173304F210D304F21C8
:10065000ED0164000F306D028A110A1203183A2B63
:100660008A110A128A110A16E8208A110A12ED0A62
:10067000031D292B85108316851083126511073001
:10068000BA008030B8003C08AA003D08AB00AE01BB
:10069000AF013E304F21051183160511831264000E
:1006A00085194F2B0730BA004030B8003C08AA002B
:1006B0003D08AB008830AC001330AD00DD20031CDA
:1006C0004F2BE3000730BA008030B8003C08AA0086
:1006D0003D08AB00AE01AF0163084F21051583163D
:1006E000051164000630831263028A150A16031C82
:1006F0007C2D8A110A12FF30E200FF30A200A20A0C
:100700002208273C8A110A12031CC12B8A110A12E3
:100710008A110A1295238A110A126302031D7F2B84
:100720002208E2008A110A12C12B03308A00220833
:1007300082074634423452344C34483453345534AE
:100740004D344E344B345A34513454345734563477
:1007500070345034643444346F344F34633443342D
:100760006734733472346D346C346E347634773469
:10077000683430343134323433343434353436340C
:100780003F346208A100273C8A110A12031C512C35
:100790008A110A12A10D8A110A12DA238A110A1289
:1007A000A00021108A110A12DA238A110A128A0083
:0C07B0002008820004308A002108002C80
:1008000082070A343F340A3489340A34D3340B342F
:100810000C340934CF34093485340A3438340B3479
:1008200045340934AB3403343A34033428340734C0
:10083000553407345834073405340634F734083453
:1008400070340834773408347E34083485340834FE
:100850008C340834933408349A340834A13408347E
:10086000E23407345B34073483340734AB34073461
:10087000D3340734FB3406347E340734153406345D
:100880004434043460340434603404346034043454
:100890006034043460340434603404346034043428
:1008A000D1340730BA008030B8003C08AA003D08B7
:1008B000AB00AE01AF010D304F213F304F213E2B39
:1008C0000730BA004030B8003C08AA003D08AB0031
:1008D0008830AC001330AD00DD20031C3E2BE3005C
:1008E0000730BA008030B8003C08AA003D08AB00D1
:1008F000AE01AF0163084F21FF30F100FF30A200CD
:10090000A20A2208023C8A110A12031C9D2C8A1199
:100910000A128A110A1296248A110A126302031D0E
:10092000802C2208F1008A110A129D2C04308A00C2
:100930002208820766346D34623464007108FF3C1B
:100940000319512CF8012030E2026208A100063C94
:100950008A110A12031CD02C8A110A12A10D8A11C5
:100960000A12BE248A110A12A00021108A110A124A
:10097000BE248A110A128A002008820004308A00EC
:10098000210882070B344D340B3484340B34BC34CF
:100990000B34F4340C342C340C3464340C349C3468
:1009A0003E2B0730BA004030B8003C08AA003D0892
:1009B000AB008830AC001330AD00DD20031C3E2BB3
:1009C000E3000730BA008030B8003C08AA003D08B8
:1009D000AB00AE01AF0163084F21FF30E200FF30F2
:1009E000A200A20A2208063C8A110A12031C122D38
:1009F0008A110A128A110A1207258A110A12630241
:100A0000031DF12C2208E2008A110A12122D053072
:100A10008A00220882076734733472346D346C3470
:100A20006E3476346208A100063C8A110A12031C57
:100A30003D2D8A110A12A10D8A110A122B258A1145
:100A40000A12A00021108A110A122B258A110A12FB
:100A50008A002008820005308A00210882070534B8
:100A60003E3405347F34053495340534AB340534D5
:100A7000C1340534D73406342B343E2B0C30ED0012
:100A80008A110A16BC208A110A120730BA00803077
:100A9000B8003C08AA003D08AB00AE01AF016C30C5
:100AA0004F213D304F21A9017108A400A5014E300E
:100AB000B0000130B1009D210D304F210D30ED000F
:100AC0008A110A16BC208A110A120730BA00803037
:100AD000B8003C08AA003D08AB00AE01AF0167308A
:100AE0004F213D304F21A9017108A400A5014E30CE
:100AF000B0000130B1009D210D304F213E2B073059
:100B0000BA008030B8003C08AA003D08AB00AE0136
:100B1000AF01A9016E08A400A5014E30B00001305C
:100B2000B1009D210D304F213E2B0730BA0080309F
:100B3000B8003C08AA003D08AB00AE01AF01A90116
:100B40006908A400A5014E30B0000130B1009D211C
:100B50000D304F213E2B0730BA008030B8003C08E2
:100B6000AA003D08AB00AE01AF01A9017008A400C6
:100B7000A5014E30B0000130B1009D210D304F2154
:100B80003E2B0730BA008030B8003C08AA003D0870
:100B9000AB00AE01AF01A9016A08A400A5014E3067
:100BA000B0000130B1009D210D304F213E2B0730A8
:100BB000BA008030B8003C08AA003D08AB00AE0186
:100BC000AF010D304F216E304F2165304F21753010
:100BD0004F2174304F2172304F2161304F216C30E2
:100BE0004F210D304F21ED0164000C306D028A1150
:100BF0000A1203182A2E8A110A1201306D07B20058
:100C000021300318013EB3003208E121F100073022
:100C1000BA008030B8003C08AA003D08AB00AE0125
:100C2000AF01A9016D08A400A5014E30B00001304C
:100C3000B1009D2120304F21A9017108A400A50118
:100C40004E30B0000130B1009D210D304F21ED0A32
:100C5000031DF42D3E2B1430F7210730BA008030ED
:100C6000B8003C08AA003D08AB000230AE00AF015E
:100C7000A9012A30A400A5014E30B0000130B10016
:100C80009D210D304F213E2B0730BA004030B80077
:100C90003C08AA003D08AB008830AC001330AD0022
:100CA000A901DD30B000B1011021031C3E2BC600AC
:100CB0002508C7000730BA008030B8003C08AA00F9
:100CC0003D08AB00AE01AF01A9014608A4004708EA
:100CD000A5004E30B0000130B1009D214608A600AD
:100CE0004708A7006430A200A3017022B2002508C3
:100CF000B3003308A3003208F8213E2B0730BA00B6
:100D00004030B8003C08AA003D08AB008830AC0079
:100D10001330AD00A901DD30B000B1011021031C7A
:100D20003E2BC4002508C5000730BA008030B8004B
:100D30003C08AA003D08AB00AE01AF01A901440880
:100D4000A4004508A5004E30B0000130B1009D213F
:100D50000730BA004030B8003C08AA003D08AB009C
:100D60008830AC001330AD00A901DD30B000B10116
:100D70001021031C3E2BC6002508C7000730BA000F
:100D80008030B8003C08AA003D08AB00AE01AF01BE
:100D9000A9014608A4004708A5004E30B000013064
:100DA000B1009D214408A6004508A7000A30A20012
:100DB000A3017022C4002508C5004608A600470804
:100DC000A7000A30A200A3017022C6002508C700B0
:100DD0000630BA000830B8004608BB004708B90022
:100DE0004508A700A5004408A60068203E2B063051
:100DF000BA000830B8006430BB00B9010F30A7005A
:100E0000A500A030A60068203E2B8A150A12642790
:100E10008A110A124008A0004108A100FF30A30077
:100E2000FF304222031D052F3E2B0730BA00403011
:100E3000B8003C08AA003D08AB008830AC00133075
:100E4000AD00A901DD30B000B1011021031C3E2B23
:100E5000ED000730BA008030B8003C08AA003D0819
:100E6000AB00AE01AF01A9016D08A400A5014E3091
:100E7000B0000130B1009D218A150A12C9278A11DC
:100E80000A12403084006D08003E4C200030031DE3
:100E90000130B200B3013208A0003308A100A30161
:100EA00000303922031D3C2F3E2B5130E8003E2BF1
:100EB0005430E8003E2B0730BA004030B8003C0800
:100EC000AA003D08AB008830AC001330AD00A9018A
:100ED000DD30B000B1011021031C3E2BEE000730C5
:100EE000BA008030B8003C08AA003D08AB00AE0153
:100EF000AF01A9016E08A400A5014E30B000013079
:100F0000B1009D213E2B0730BA004030B8003C08AC
:100F1000AA003D08AB008830AC001330AD00A90139
:100F2000DD30B000B1011021031C3E2BE900073079
:100F3000BA008030B8003C08AA003D08AB00AE0102
:100F4000AF01A9016908A400A5014E30B00001302D
:100F5000B1009D213E2B0730BA004030B8003C085C
:100F6000AA003D08AB008830AC001330AD00A901E9
:100F7000DD30B000B1011021031C3E2BF000073022
:100F8000BA008030B8003C08AA003D08AB00AE01B2
:100F9000AF01A9017008A400A5014E30B0000130D6
:100FA000B1009D213E2B0730BA004030B8003C080C
:100FB000AA003D08AB008830AC001330AD00A90199
:100FC000DD30B000B1011021031C3E2BEA000730D8
:100FD000BA008030B8003C08AA003D08AB00AE0162
:100FE000AF01A9016A08A400A5014E30B00001308C
:100FF000B1009D213E2B0F30ED000730BA0040308C
:10100000B8003C08AA003D08AB008830AC001330A3
:10101000AD00A901DD30B000B1018A158A1110219F
:101020008A158A11031C3E2B8A15ED000730BA0081
:101030008030B8003C08AA003D08AB00AE01AF010B
:10104000A9016D08A400A5014E30B0000130B10027
:101050008A119D218A150730BA004030B8003C083B
:10106000AA003D08AB008830AC001330AD00A901E8
:10107000DD30B000B1018A1110218A158A11031CDC
:101080003E2B8A15F1000730BA008030B8003C08CA
:10109000AA003D08AB00AE01AF01A9017108A40090
:1010A000A5014E30B0000130B1008A119D218A1592
:1010B00064000C306D028A1103183E2B8A15013032
:1010C0006D07B20021300318013EB3003208031748
:1010D0008D00031371088A11E9218A158A113E2BAC
:1010E0000C30ED001030EC008A150A12C7280C30C5
:1010F000ED004030EC008A150A12C7280C30ED00D4
:101100001030EC008A150A12A8280C30ED0040308F
:10111000EC008A150A12A8280D30ED001030EC0002
:101120008A150A12A8280D30ED004030EC008A150F
:101130000A12A8280D30ED001030EC008A150A12B2
:10114000C7280D30ED004030EC008A150A12C72880
:101150008A110A16BC208A150A1271086C07B2009F
:10116000B301B30DFF30A000A1013308A300320882
:101170008A111E228A15F1008514831685108A159E
:101180000A12831218278A150A128A113E2B8A1115
:101190000A16BC208A150A127108A0006C088A1170
:1011A00019228A15B200B3016C083202F1008514CD
:1011B000831685108A150A12831218278A150A12B7
:1011C0008A113E2B05118316051107308312BA00D0
:1011D0004030B8003C08AA003D08AB008830AC00A5
:1011E0001330AD00A901DD30B000B1018A1110212A
:1011F0008A158A11031C3E2B8A15F3000730BA00AA
:101200008030B8003C08AA003D08AB00AE01AF0139
:10121000A9017308A400A5014E30B0000130B1004F
:101220008A119D218A150730BA004030B8003C0869
:10123000AA003D08AB008830AC001330AD00A90116
:10124000DD30B000B1018A1110218A158A11031C0A
:101250003E2B8A15F2000730BA008030B8003C08F7
:10126000AA003D08AB00AE01AF01A9017208A400BD
:10127000A5014E30B0000130B1008A119D218A15C0
:10128000051583160511640083127308003C8A1546
:101290000A12031965298A150A120C30ED00640040
:1012A0007308FF3C8A150A12031D60298A150A1269
:1012B0008A110A16E8208A150A128A150A12652967
:1012C0008A150A1218278A150A1264007208003C4F
:1012D0008A1103193E2B8A150D30ED006400720847
:1012E000FF3C8A150A12031D7E298A150A128A11EB
:1012F0000A16E8208A150A128A113E2B8A150A124C
:1013000018278A150A128A113E2B0130ED0064005D
:101310000C306D028A150A120318A5298A150A12C3
:1013200001306D07B20021300318013EB3003208CE
:101330008A11E1218A15F1008A150A1218278A15E7
:101340000A120230ED07031C8729C2012130C300B5
:101350008A150A12D02EED0164000C306D028A1538
:101360000A120318C9298A150A1201306D07B20042
:1013700021300318013EB30032088A11E1218A1599
:10138000F1008A150A1218278A150A12ED0A031DA0
:10139000AC29C2012130C3008A150A12D02E65156E
:1013A000ED0164000C306D028A150A120318342A0C
:1013B0008A150A128A110A164F208A150A12043059
:1013C0006407E30074088A115E208A1566088A1192
:1013D00063208A155430AA004030AB00AE01AF0143
:1013E00063088A1149218A1500308A1149218A151A
:1013F00074088A115E208A155430AA004030AB0070
:10140000F430AC000130AD008A11DD208A15031CD8
:10141000E229F1006E08A000A10104308A112A22FD
:101420008A15B2002108B3000030B2070318B30ACE
:1014300064083207E30074088A115E208A15660882
:101440008A1163208A155430AA004030AB00AE01E7
:10145000AF0163088A1149218A1571088A1149214F
:101460008A15ED0A031DD129FF30C0040F30C104D5
:101470007730C2002130C3008A150A12D42C003004
:1014800065180130F10064008A150A12E51C4C2A27
:101490008A150A120230F1077108A200033C8A156E
:1014A0000A12031C852A8A150A120310220DA207AC
:1014B0008A150A1275228A150A12A000A20A8A1534
:1014C0000A1275228A150A12A100A20A8A150A12A6
:1014D00075228A150A128A11C4208A152008C200B2
:1014E0002108C3008A150A12852A0A308A002208B8
:1014F00082078C34213400347F3421340034863424
:1015000021340034793421340034E5108A150A126C
:10151000D42C003065180130F10064008A150A12DD
:10152000E51C962A8A150A120230F1077108A200FA
:10153000033C8A150A12031CCF2A8A150A120310CB
:10154000220DA2078A150A12BF228A150A12A000CC
:10155000A20A8A150A12BF228A150A12A100A20A3B
:101560008A150A12BF228A150A128A11C4208A1506
:101570002008C2002108C3008A150A12CF2A0A30A7
:101580008A0022088207993421340034A634213499
:101590000034933421340034A03421340034E51075
:1015A0008A150A12D42C003065180130A200013CC3
:1015B0008A150A12031C082B8A150A120310220D21
:1015C000A2078A150A12FE228A150A12A000A20A90
:1015D0008A150A12FE228A150A12A100A20A8A1589
:1015E0000A12FE228A150A128A11C4208A152008BE
:1015F000C2002108C3008A150A12082B0B308A008A
:1016000022088207AD3421340034B434213400344C
:10161000E5148A150A12D42C003065180130A20096
:10162000013C8A150A12031C412B8A150A12031069
:10163000220DA2078A150A1237238A150A12A00062
:10164000A20A8A150A1237238A150A12A100A20AD1
:101650008A150A1237238A150A128A11C4208A159C
:101660002008C2002108C3008A150A12412B0B3042
:101670008A0022088207BB3421340034C23421346A
:101680000034E5148A150A12D42CC930C200213066
:10169000C300E5108A150A12D42C7108A100023C7F
:1016A0008A150A12031C702B8A150A12A10D8A15BD
:1016B0000A1266238A150A12A00021108A150A123E
:1016C00066238A150A128A00200882000B308A00DD
:1016D000210882070B3470340B3476340B347D349C
:1016E000C201F130C3008A150A12D42C0130C200A5
:1016F000F130C3008A150A12D42C0230C200F13036
:10170000C3008A150A12D42C7108A100023C8A1564
:101710000A12031CA72B8A150A12A10D8A150A1298
:101720009D238A150A12A00021108A150A129D23F2
:101730008A150A128A00200882000B308A002108CC
:1017400082070B34A7340B34AE340B34B53403307A
:10175000C200F130C3008A150A12D42C0430C20032
:10176000F130C3008A150A12D42C0530C200F130C2
:10177000C3008A150A12D42C7108A100023C8A15F4
:101780000A12031CDF2B8A150A12A10D8A150A12F0
:10179000D5238A150A12A00021108A150A12D52312
:1017A0008A150A128A00200882000B308A0021085C
:1017B00082070B34DF340B34E6340B34ED3406305F
:1017C000C200F130C3008A150A12D42C0730C200BF
:1017D000F130C3008A150A12D42C0830C200F1304F
:1017E000C3008A150A12D42C7108A100023C8A1584
:1017F0000A12031C172C8A150A12A10D8A150A1247
:101800000D248A150A12A00021108A150A120D242F
:101810008A150A128A00200882000C308A002108EA
:1018200082070C3417340C341E340C342534093040
:10183000C200F130C3008A150A12D42C0A30C2004B
:10184000F130C3008A150A12D42C0B30C200F130DB
:10185000C3008A150A12D42C7108A100023C8A1513
:101860000A12031C4F2C8A150A12A10D8A150A129E
:1018700045248A150A12A00021108A150A1245244F
:101880008A150A128A00200882000C308A0021087A
:1018900082070C344F340C3456340C345D340C3025
:1018A000C200F130C3008A150A12D42C0D30C200D8
:1018B000F130C3008A150A12D42C0E30C200F13068
:1018C000C3008A150A12D42C7108A100023C8A15A3
:1018D0000A12031C872C8A150A12A10D8A150A12F6
:1018E0007D248A150A12A00021108A150A127D246F
:1018F0008A150A128A00200882000C308A0021080A
:1019000082070C3487340C348E340C3495340F3009
:10191000C200F130C3008A150A12D42C1030C20064
:10192000F130C3008A150A12D42C1130C200F130F4
:10193000C3008A150A12D42C7108A100023C8A1532
:101940000A12031CBF2C8A150A12A10D8A150A124D
:10195000B5248A150A12A00021108A150A12B5248E
:101960008A150A128A00200882000C308A00210899
:1019700082070C34BF340C34C6340C34CD341230EE
:10198000C200F130C3008A150A12D42C1330C200F1
:10199000F130C3008A150A12D42C1430C200F13081
:1019A000C3008A150A12D42C64008A150A128518FD
:1019B000E32C8A150A1264308A11F7218A158514DE
:1019C0008316851083124208A0004308A100F0305E
:1019D000A30000308A113F228A158A150A12031DBE
:1019E000FB2C8A150A128A110A1603218A150A127B
:1019F0008A150A12042D42088A11E1218A15BE00B7
:101A0000BF01C20A0319C30A3E08A0003F08A10093
:101A1000A30100308A1139228A158A11031D3E2B39
:101A20008A153E08A0003F08A100F030A300003056
:101A30008A113F228A158A150A12031D2B2D8A1539
:101A40000A128A110A16B2268A150A127108ED00C6
:101A50008A150A12332D3E088A11E1218A15ED00FC
:101A6000BE0A0319BF0A64006D080F3C8A150A12EA
:101A70000319A02E8A150A123E08A0003F08A100F3
:101A8000F030A30000308A113F228A158A150A120D
:101A9000031D542D8A150A128A110A16B2268A15B8
:101AA0000A128A150A125C2D3E088A11E1218A1554
:101AB000F100BE0A0319BF0A6400023071028A15E0
:101AC0000A120318792D8A150A1264006808543C1A
:101AD0000319D42C64007108013C8A150A120319F9
:101AE000762D8A150A127130E800D42C6630E80091
:101AF000D42C64006D08003C8A150A12031DA22D27
:101B00008A150A12FF30A200A20A2208013C8A1597
:101B10000A12031CA22D8A150A128A150A129C2584
:101B20008A150A127102031D842D22186514221CC5
:101B300065108A150A12A22D0D308A00220882072C
:101B4000FF34023464008A150A126D1C2F2E8A1588
:101B50000A1201306D07B20021300318013EB300B4
:101B600032088A11E1218A15EB00640006306D020B
:101B70008A150A120318F22D8A150A1264007108D8
:101B8000023C8A150A120319E42D8A150A126B0801
:101B9000A00069088A1119228A15B200B3016908E8
:101BA000B202031CB3036A08B2070318B30AFF307A
:101BB000A000A1013308A30032088A111E228A1551
:101BC000F1008A150A129A2E6B08A00069088A1182
:101BD00019228A15B200B30169083202F1008A1590
:101BE0000A129A2E64007108FF3C8A150A12031922
:101BF0001D2E8A150A126B086907B200B301B30DD6
:101C0000FF30A000A1013308A30032088A111E2270
:101C10008A15B2002108B3003208A0003308A100E1
:101C20006A088A111A228A15B2002108B3006A08CC
:101C30003202F1008A150A129A2E6B086907B20067
:101C4000B301B30DFF30A000A1013308A300320897
:101C50008A111E228A15F1008A150A129A2E013065
:101C60006D07B20021300318013EB30032088A111B
:101C7000E1218A15EB00640071087F3C8A150A1285
:101C8000031D542E8A150A126B08F10064006D08BA
:101C9000003C8A150A12031D9A2E8A150A126B0837
:101CA000E7008A150A129A2E640071086B028A15E1
:101CB0000A12031C772E8A150A126B08A0007008FE
:101CC0008A1119228A15B200B30170083202F1009C
:101CD00064006D08003C8A150A12031D9A2E8A15AD
:101CE0000A1271086A07E7008A150A129A2E6B0811
:101CF0007007B200B301B30DFF30A000A10133089B
:101D0000A30032088A111E228A15F10064006D08B2
:101D1000003C8A150A12031D9A2E8A150A127108B0
:101D2000A0006A088A1119228A15B200B3016A0854
:101D30003202E7008A150A1218278A150A12112D95
:101D400064008A150A126519D02E8A150A12073006
:101D5000BA004030B8003C08AA003D08AB0064302F
:101D6000AC00AD018A11DD208A158A150A12031C08
:101D7000BC2E8A150A12E300003085190130A0003C
:101D800001308A1137228A15B2006308A00048305A
:101D90008A1137228A15B40032083404031DCF2972
:101DA00064006808713C0319D42C6808A000543002
:101DB0008A1137228A15B2006808A00051308A11B2
:101DC00037228A15B400320834048A150A12031D1A
:101DD000F92E8A150A128A110A160F208A150A127C
:101DE00064006708FF3C8A150A120319152F8A152B
:101DF0000A128A150A1264278A150A12FF30400552
:101E0000B2000F304105B3003208A0003308A10032
:101E10000F30A300FF308A1142228A15031DA02E25
:101E200064006808543C0319D42C5130E800D42CC9
:101E3000FF30A000A10171088A111D228A15B2008D
:101E40002108B3000230A000A1013308A30032082A
:101E50008A111B228A15F100403084006D08003E73
:101E60008A114C208A1503108A1157208A158A116D
:101E70000A164F208A150A126E08A000A10104302C
:101E80008A112A228A15B2002108B3000030B20755
:101E90000318B30A64083207E30074088A115E204D
:101EA0008A1566088A1163208A155430AA004030CA
:101EB000AB00AE01AF0163088A1149218A15710890
:101EC0008A1149218A150800ED0164000D306D0268
:101ED0008A150A120318C72F8A150A128A110A16C0
:101EE0004F208A150A1274088A115E208A15660826
:101EF0008A1163208A155430AA004030AB00AE012D
:101F0000AF0108308A1149218A1500308A11492110
:101F10008A1574088A115E208A155430AA00403050
:101F2000AB003230AC00AD018A11DD208A15031CF4
:101F3000732FEF00E4016400033064028A150A1273
:101F40000318C32F8A150A126D086407B400B5017F
:101F5000B50D6F3084006408003E8A114C208A154C
:101F60000030031D0130B200B3014030840034085A
:101F7000003E8A114C208A15320C8A1157208A158E
:101F8000E40A031D9B2F0330ED07031C652FC117C7
:101F900008008A110A164F208A150A1274088A113D
:101FA0005E208A1566088A1163208A155430AA00BB
:101FB0004030AB00AE01AF0108308A1149218A15CB
:101FC00000308A1149218A1574088A115E208A1509
:101FD0005430AA004030AB003230AC00AD018A1161
:101FE000DD208A15031CCE2FEF006F3084006408BB
:101FF000003E8A114C208A150030031D0130B200CA
:10200000B301403084006D08003E8A110A160A129E
:102010004C200A16320C0A1257200A160800ED014D
:102020008A110A16BC208A110A1600306518013080
:10203000A100013C8A110A16031C38288A110A16CD
:10204000A10D8A110A1630208A110A16A00021104B
:102050008A110A1630208A110A168A002008820086
:1020600010308A002108820710343834103442348A
:102070006400670871028A110A1603184C288A1135
:102080000A1608006400710867028A110A1603180C
:102090004C288A110A160800FF30E70008006D0876
:1020A0000E3C8A110A16031C73288A110A168A111B
:1020B0000A1660208A110A16E4008A110A1673288B
:1020C00010308A006D088207023401340034023473
:1020D0000134003400340134023400340134023459
:1020E0000234013400346D080E3C8A110A16031CB8
:1020F00097288A110A168A110A1684208A110A164C
:10210000F4008A110A16972810308A006D08820799
:102110000A340A340A3408340834083400340034E9
:1021200000340C340C340C340434043404346D089E
:102130000E3C8A110A16031CBB288A110A168A1142
:102140000A16A8208A110A16E6008A110A16BB2868
:1021500010308A006D0882070B340B340B340934BD
:10216000093409340134013401340D340D340D3493
:1021700005340534053408004F2004306407E300BB
:1021800074080A125E200A1666080A1263200A16EC
:102190005430AA004030AB00AE01AF0163080A1210
:1021A00049210A1671080A1249210A1674080A12EE
:1021B0005E200A165430AA004030AB003230AC002A
:1021C000AD010A12DD200A16031CC028F100080028
:1021D0004F200C306407E30074080A125E200A16D0
:1021E00066080A1263200A165430AA004030AB0079
:1021F000AE01AF0163080A1249210A1600300A1223
:1022000049210A16080000304202B2000130031CC6
:10221000013E4302B30000303202F6007608A1000E
:10222000143C8A110A16031C55298A110A16A10D9D
:102230008A110A1627218A110A16A00021108A1174
:102240000A1627218A110A168A00200882001130F6
:102250008A00210882071134583411349134113422
:10226000CA341234033412344534123487341234ED
:10227000C934133416341334583413349A341334A1
:10228000DC3414341E34143460341434A234143462
:10229000E43415342634153468341534AA3415342E
:1022A000EC3416342E3416347034BE01BF010800ED
:1022B0007808A200023C8A110A16031C8E298A1192
:1022C0000A160310220DA2078A110A1681218A110B
:1022D0000A16A000A20A8A110A1681218A110A167A
:1022E000A100A20A8A110A1681218A110A160A126D
:1022F000C4200A162008BE002108BF008A110A1651
:102300008E2911308A0022088207113421340034CA
:102310000034F1340034003400340034F701F80A9A
:1023200008007808A200023C8A110A16031CC7297B
:102330008A110A160310220DA2078A110A16BA2161
:102340008A110A16A000A20A8A110A16BA218A1155
:102350000A16A100A20A8A110A16BA218A110A16BF
:102360000A12C4200A162008BE002108BF008A11E4
:102370000A16C72911308A00220882071134213435
:1023800000340134F1340034003400340034F701F7
:10239000F80A08007808A200023C8A110A16031CF9
:1023A000002A8A110A160310220DA2078A110A16A2
:1023B000F3218A110A16A000A20A8A110A16F32133
:1023C0008A110A16A100A20A8A110A16F3218A119B
:1023D0000A160A12C4200A162008BE002108BF00EF
:1023E0008A110A16002A11308A0022088207113445
:1023F000213400340234F134003400340034003429
:10240000F701F80A08007808A200053C8A110A16AC
:10241000031C422A8A110A160310220DA2078A11F0
:102420000A162C228A110A16A000A20A8A110A167C
:102430002C228A110A16A100A20A8A110A162C223D
:102440008A110A160A12C4200A162008BE002108A2
:10245000BF008A110A16422A12308A002208820717
:102460007334213400340334F134003475342134AE
:1024700000340434F1340034113421340034003495
:1024800000340034F701F80A08007808A200053C7F
:102490008A110A16031C842A8A110A160310220DB7
:1024A000A2078A110A166E228A110A16A000A20A31
:1024B0008A110A166E228A110A16A100A20A8A112E
:1024C0000A166E228A110A160A12C4200A16200859
:1024D000BE002108BF008A110A16842A12308A0021
:1024E000220882077334213400340334F134003479
:1024F0007534213400340534F1340034113421347E
:102500000034003400340034F701F80A0800780879
:10251000A200053C8A110A16031CC62A8A110A1653
:102520000310220DA2078A110A16B0228A110A1678
:10253000A000A20A8A110A16B0228A110A16A10066
:10254000A20A8A110A16B0228A110A160A12C42097
:102550000A162008BE002108BF008A110A16C62AE2
:1025600012308A0022088207733421340034033485
:10257000F13400347534213400340634F13400343D
:10258000113421340034003400340034F701F80AE7
:1025900008007808A200053C8A110A16031C132BB8
:1025A0008A110A160310220DA2078A110A16F222B6
:1025B0008A110A16A000A20A8A110A16F2228A11AA
:1025C0000A16A100A20A8A110A16F2228A110A1614
:1025D0000A12C4200A162008BE002108BF008A1172
:0C25E0000A16132B13308A002208002B6F
:1026000082077334213400340734F13400347534D4
:10261000213400340834F1340034113421340034CE
:10262000003400340034F701F80A08007808A200EA
:10263000053C8A110A16031C552B8A110A16031031
:10264000220DA2078A110A163F238A110A16A0003A
:10265000A20A8A110A163F238A110A16A100A20AA9
:102660008A110A163F238A110A160A12C4200A1672
:102670002008BE002108BF008A110A16552B13300E
:102680008A00220882077334213400340734F1347D
:1026900000347534213400340934F13400341134F9
:1026A00021340034003400340034F701F80A080003
:1026B0007808A200053C8A110A16031C972B8A1180
:1026C0000A160310220DA2078A110A1681238A1105
:1026D0000A16A000A20A8A110A1681238A110A1674
:1026E000A100A20A8A110A1681238A110A160A1267
:1026F000C4200A162008BE002108BF008A110A164D
:10270000972B13308A002208820773342134003457
:102710000734F13400347534213400340A34F13490
:102720000034113421340034003400340034F70113
:10273000F80A08007808A200053C8A110A16031C52
:10274000D92B8A110A160310220DA2078A110A1624
:10275000C3238A110A16A000A20A8A110A16C323EB
:102760008A110A16A100A20A8A110A16C3238A1125
:102770000A160A12C4200A162008BE002108BF004B
:102780008A110A16D92B13308A0022088207733463
:10279000213400340B34F1340034753421340034E6
:1027A0000C34F1340034113421340034003400345A
:1027B0000034F701F80A08007808A200053C8A11E5
:1027C0000A16031C1B2C8A110A160310220DA207DD
:1027D0008A110A1605248A110A16A000A20A8A1173
:1027E0000A1605248A110A16A100A20A8A110A16DD
:1027F00005248A110A160A12C4200A162008BE00EF
:102800002108BF008A110A161B2C14308A002208E6
:1028100082077334213400340B34F13400347534BE
:10282000213400340D34F1340034113421340034B7
:10283000003400340034F701F80A08007808A200D8
:10284000053C8A110A16031C5D2C8A110A16031016
:10285000220DA2078A110A1647248A110A16A0001F
:10286000A20A8A110A1647248A110A16A100A20A8E
:102870008A110A1647248A110A160A12C4200A1657
:102880002008BE002108BF008A110A165D2C1430F2
:102890008A00220882077334213400340B34F13467
:1028A00000347534213400340E34F13400341134E2
:1028B00021340034003400340034F701F80A0800F1
:1028C0007808A200053C8A110A16031C9F2C8A1165
:1028D0000A160310220DA2078A110A1689248A11EA
:1028E0000A16A000A20A8A110A1689248A110A1659
:1028F000A100A20A8A110A1689248A110A160A124C
:10290000C4200A162008BE002108BF008A110A163A
:102910009F2C14308A00220882077334213400343B
:102920000F34F13400347534213400341034F13470
:102930000034113421340034003400340034F70101
:10294000F80A08007808A200053C8A110A16031C40
:10295000E12C8A110A160310220DA2078A110A1609
:10296000CB248A110A16A000A20A8A110A16CB24C7
:102970008A110A16A100A20A8A110A16CB248A110A
:102980000A160A12C4200A162008BE002108BF0039
:102990008A110A16E12C14308A0022088207733447
:1029A000213400340F34F1340034753421340034D0
:1029B0001134F13400341134213400340034003443
:1029C0000034F701F80A08007808A200053C8A11D3
:1029D0000A16031C232D8A110A160310220DA207C2
:1029E0008A110A160D258A110A16A000A20A8A1158
:1029F0000A160D258A110A16A100A20A8A110A16C2
:102A00000D258A110A160A12C4200A162008BE00D3
:102A10002108BF008A110A16232D15308A002208CA
:102A200082077334213400340F34F13400347534A8
:102A3000213400341234F1340034113421340034A0
:102A4000003400340034F701F80A08007808A200C6
:102A5000053C8A110A16031C652D8A110A160310FB
:102A6000220DA2078A110A164F258A110A16A00004
:102A7000A20A8A110A164F258A110A16A100A20A73
:102A80008A110A164F258A110A160A12C4200A163C
:102A90002008BE002108BF008A110A16652D1530D6
:102AA0008A00220882077334213400341334F1344D
:102AB00000347534213400341434F13400341134CA
:102AC00021340034003400340034F701F80A0800DF
:102AD0007808A200053C8A110A16031CA72D8A114A
:102AE0000A160310220DA2078A110A1691258A11CF
:102AF0000A16A000A20A8A110A1691258A110A163E
:102B0000A100A20A8A110A1691258A110A160A1230
:102B1000C4200A162008BE002108BF008A110A1628
:102B2000A72D15308A00220882077334213400341F
:102B30001334F13400347534213400341534F13455
:102B40000034113421340034003400340034F701EF
:102B5000F80A08007808A200053C8A110A16031C2E
:102B6000E92D8A110A160310220DA2078A110A16EE
:102B7000D3258A110A16A000A20A8A110A16D325A3
:102B80008A110A16A100A20A8A110A16D3258A11EF
:102B90000A160A12C4200A162008BE002108BF0027
:102BA0008A110A16E92D15308A002208820773342B
:102BB000213400341334F1340034753421340034BA
:102BC0001634F1340034113421340034003400342C
:102BD0000034F701F80A08007808A200053C8A11C1
:102BE0000A16031C2B2E8A110A160310220DA207A7
:102BF0008A110A1615268A110A16A000A20A8A113D
:102C00000A1615268A110A16A100A20A8A110A16A6
:102C100015268A110A160A12C4200A162008BE00B8
:102C20002108BF008A110A162B2E16308A002208AE
:102C300082077334213400341734F134003475348E
:102C4000213400341834F134003411342134003488
:102C5000003400340034F701F80A08007808A200B4
:102C6000053C8A110A16031C6D2E8A110A160310E0
:102C7000220DA2078A110A1657268A110A16A000E9
:102C8000A20A8A110A1657268A110A16A100A20A58
:102C90008A110A1657268A110A160A12C4200A1621
:102CA0002008BE002108BF008A110A166D2E1630BA
:102CB0008A00220882077334213400341734F13437
:102CC00000347534213400341934F13400341134B3
:102CD00021340034003400340034F701F80A0800CD
:102CE0007808A200053C8A110A16031CAF2E8A112F
:102CF0000A160310220DA2078A110A1699268A11B4
:102D00000A16A000A20A8A110A1699268A110A1622
:102D1000A100A20A8A110A1699268A110A160A1215
:102D2000C4200A162008BE002108BF008A110A1616
:102D3000AF2E16308A002208820773342134003403
:102D40001734F13400347534213400341A34F1343A
:102D50000034113421340034003400340034F701DD
:102D6000F80A080000303E02B2000130031C013EA8
:102D70003F02B30000303202F5007508A1001A3C92
:102D80008A110A16031C372F8A110A16A10D8A11FF
:102D90000A16D6268A110A16A00021108A110A16D0
:102DA000D6268A110A168A002008820017308A0067
:042DB0002108002FC7
:102E0000820717343A3417348E341734E2341834C6
:102E10003934183471341834A9341834E13419347D
:102E2000193419345134193489341934C1341934EA
:102E3000F9341A3431341A3469341A34A1341A3456
:102E4000D9341B3411341B3449341B3481341B34C2
:102E5000B9341B34F1341C3429341C3461341C342F
:102E600099341C34D1341D340C341D3444340F30A7
:102E7000ED0008007708A2000C3C8A110A16031C1A
:102E80008C2F8A110A160310220DA2078A110A1626
:102E900061278A110A16A000A20A8A110A16612760
:102EA0008A110A16A100A20A8A110A1661278A113C
:102EB0000A160A12C4200A162008F1008A110A16FE
:102EC0008C2F17308A002208820700340034003427
:102ED000023400340034023400340034023400344C
:102EE0000034043400340034023400340034063436
:102EF00000340034FF34003400340834003400342B
:102F0000FF34003400340A3400340034FF34003419
:102F100000340F3400340034F70A08007708A200A8
:102F20000C3C8A110A16031CE02F8A110A160310A2
:102F3000220DA2078A110A16B5278A110A16A000C7
:102F4000A20A8A110A16B5278A110A16A100A20A36
:102F50008A110A16B5278A110A160A12C4200A16FF
:102F60002008F1008A110A16E02F17308A00220883
:102F700082070034003400347F34003400340234DB
:102F8000003400347F34003400340434003400341E
:102F90007F34003400340634003400347F3400348D
:102FA00000340834003400347F34003400340A34F0
:102FB000003400347F34003400340F3400340034E3
:102FC000F70A08007708A2000C3C8A150A16031CB1
:102FD00037288A110A160310220DA2078A150A162D
:102FE0000C208A110A16A000A20A8A150A160C20C3
:102FF0008A110A16A100A20A8A150A160C208A1143
:103000000A168A158A110A12C4208A150A1620087F
:10301000F1008A150A16372818308A00220882071C
:10302000003400340034FF340034003402340034FF
:103030000034FF3400340034043400340034FF34EE
:1030400000340034063400340034023400340034D8
:103050000834003400340234003400340A340034BC
:1030600000340234003400340F3400340034F70AE2
:1030700008007708A200023C8A150A16031C6F2874
:103080008A150A160310220DA2078A150A16622055
:103090008A150A16A000A20A8A150A1662208A1545
:1030A0000A16A100A20A8A150A1662208A150A16B3
:1030B0008A110A12C4208A150A162008F1008A15FE
:1030C0000A166F2818308A0022088207013400345B
:1030D0000034FF34003400340F3400340034F70A75
:1030E00008007708A200023C8A150A16031CA728CC
:1030F0008A150A160310220DA2078A150A169A20AD
:103100008A150A16A000A20A8A150A169A208A159C
:103110000A16A100A20A8A150A169A208A150A160A
:103120008A110A12C4208A150A162008F1008A158D
:103130000A16A72818308A002208820700340034B3
:103140000034FF34003400340F3400340034F70A04
:1031500008007708A200023C8A150A16031CDF2823
:103160008A150A160310220DA2078A150A16D22004
:103170008A150A16A000A20A8A150A16D2208A15F4
:103180000A16A100A20A8A150A16D2208A150A1662
:103190008A110A12C4208A150A162008F1008A151D
:1031A0000A16DF2818308A0022088207003400340B
:1031B00000347F34003400340F3400340034F70A14
:1031C00008007708A200023C8A150A16031C17297A
:1031D0008A150A160310220DA2078A150A160A215B
:1031E0008A150A16A000A20A8A150A160A218A154B
:1031F0000A16A100A20A8A150A160A218A150A16B9
:103200008A110A12C4208A150A162008F1008A15AC
:103210000A16172919308A00220882070034003460
:1032200000340234003400340F3400340034F70A20
:1032300008007708A200023C8A150A16031C4F29D1
:103240008A150A160310220DA2078A150A164221B2
:103250008A150A16A000A20A8A150A1642218A15A2
:103260000A16A100A20A8A150A1642218A150A1610
:103270008A110A12C4208A150A162008F1008A153C
:103280000A164F2919308A002208820707340034B1
:1032900000340234003400340F3400340034F70AB0
:1032A00008007708A200023C8A150A16031C872929
:1032B0008A150A160310220DA2078A150A167A210A
:1032C0008A150A16A000A20A8A150A167A218A15FA
:1032D0000A16A100A20A8A150A167A218A150A1668
:1032E0008A110A12C4208A150A162008F1008A15CC
:1032F0000A16872919308A0022088207063400340A
:1033000000340234003400340F3400340034F70A3F
:1033100008007708A200023C8A150A16031CBF2980
:103320008A150A160310220DA2078A150A16B22161
:103330008A150A16A000A20A8A150A16B2218A1551
:103340000A16A100A20A8A150A16B2218A150A16BF
:103350008A110A12C4208A150A162008F1008A155B
:103360000A16BF2919308A00220882070634003461
:1033700000347F34003400340F3400340034F70A52
:1033800008007708A200023C8A150A16031CF729D8
:103390008A150A160310220DA2078A150A16EA21B9
:1033A0008A150A16A000A20A8A150A16EA218A15A9
:1033B0000A16A100A20A8A150A16EA218A150A1617
:1033C0008A110A12C4208A150A162008F1008A15EB
:1033D0000A16F72919308A002208820706340034B9
:1033E0000034FF34003400340F3400340034F70A62
:1033F00008007708A200023C8A150A16031C2F2A2F
:103400008A150A160310220DA2078A150A1622220F
:103410008A150A16A000A20A8A150A1622228A15FF
:103420000A16A100A20A8A150A1622228A150A166D
:103430008A110A12C4208A150A162008F1008A157A
:103440000A162F2A1A308A00220882070334003411
:103450000034FF34003400340F3400340034F70AF1
:1034600008007708A200023C8A150A16031C672A86
:103470008A150A160310220DA2078A150A165A2267
:103480008A150A16A000A20A8A150A165A228A1557
:103490000A16A100A20A8A150A165A228A150A16C5
:1034A0008A110A12C4208A150A162008F1008A150A
:1034B0000A16672A1A308A0022088207023400346A
:1034C0000034FF34003400340F3400340034F70A81
:1034D00008007708A200023C8A150A16031C9F2ADE
:1034E0008A150A160310220DA2078A150A169222BF
:1034F0008A150A16A000A20A8A150A1692228A15AF
:103500000A16A100A20A8A150A1692228A150A161C
:103510008A110A12C4208A150A162008F1008A1599
:103520000A169F2A1A308A002208820702340034C1
:1035300000347F34003400340F3400340034F70A90
:1035400008007708A200023C8A150A16031CD72A35
:103550008A150A160310220DA2078A150A16CA2216
:103560008A150A16A000A20A8A150A16CA228A1506
:103570000A16A100A20A8A150A16CA228A150A1674
:103580008A110A12C4208A150A162008F1008A1529
:103590000A16D72A1A308A00220882070234003419
:1035A00000340234003400340F3400340034F70A9D
:1035B00008007708A200023C8A150A16031C0F2B8C
:1035C0008A150A160310220DA2078A150A1602236D
:1035D0008A150A16A000A20A8A150A1602238A155D
:1035E0000A16A100A20A8A150A1602238A150A16CB
:1035F0008A110A12C4208A150A162008F1008A15B9
:103600000A160F2B1B308A00220882070934003467
:1036100000340234003400340F3400340034F70A2C
:1036200008007708A200023C8A150A16031C472BE3
:103630008A150A160310220DA2078A150A163A23C4
:103640008A150A16A000A20A8A150A163A238A15B4
:103650000A16A100A20A8A150A163A238A150A1622
:103660008A110A12C4208A150A162008F1008A1548
:103670000A16472B1B308A002208820708340034C0
:1036800000340234003400340F3400340034F70ABC
:1036900008007708A200023C8A150A16031C7F2B3B
:1036A0008A150A160310220DA2078A150A1672231C
:1036B0008A150A16A000A20A8A150A1672238A150C
:1036C0000A16A100A20A8A150A1672238A150A167A
:1036D0008A110A12C4208A150A162008F1008A15D8
:1036E0000A167F2B1B308A00220882070834003418
:1036F00000347F34003400340F3400340034F70ACF
:1037000008007708A200023C8A150A16031CB72B92
:103710008A150A160310220DA2078A150A16AA2373
:103720008A150A16A000A20A8A150A16AA238A1563
:103730000A16A100A20A8A150A16AA238A150A16D1
:103740008A110A12C4208A150A162008F1008A1567
:103750000A16B72B1B308A0022088207083400346F
:103760000034FF34003400340F3400340034F70ADE
:1037700008007708A200023C8A150A16031CEF2BEA
:103780008A150A160310220DA2078A150A16E223CB
:103790008A150A16A000A20A8A150A16E2238A15BB
:1037A0000A16A100A20A8A150A16E2238A150A1629
:1037B0008A110A12C4208A150A162008F1008A15F7
:1037C0000A16EF2B1B308A002208820705340034CA
:1037D0000034FF34003400340F3400340034F70A6E
:1037E00008007708A200023C8A150A16031C272C41
:1037F0008A150A160310220DA2078A150A161A2422
:103800008A150A16A000A20A8A150A161A248A1511
:103810000A16A100A20A8A150A161A248A150A167F
:103820008A110A12C4208A150A162008F1008A1586
:103830000A16272C1C308A00220882070434003420
:103840000034FF34003400340F3400340034F70AFD
:1038500008007708A200023C8A150A16031C5F2C98
:103860008A150A160310220DA2078A150A16522479
:103870008A150A16A000A20A8A150A1652248A1569
:103880000A16A100A20A8A150A1652248A150A16D7
:103890008A110A12C4208A150A162008F1008A1516
:1038A0000A165F2C1C308A00220882070434003478
:1038B00000347F34003400340F3400340034F70A0D
:1038C00008007708A200023C8A150A16031C972CF0
:1038D0008A150A160310220DA2078A150A168A24D1
:1038E0008A150A16A000A20A8A150A168A248A15C1
:1038F0000A16A100A20A8A150A168A248A150A162F
:103900008A110A12C4208A150A162008F1008A15A5
:103910000A16972C1C308A002208820704340034CF
:1039200000340234003400340F3400340034F70A19
:1039300008007708A200023C8A150A16031CCF2C47
:103940008A150A160310220DA2078A150A16C22428
:103950008A150A16A000A20A8A150A16C2248A1518
:103960000A16A100A20A8A150A16C2248A150A1686
:103970008A110A12C4208A150A162008F1008A1535
:103980000A16CF2C1C308A00220882070B34003420
:1039900000340234003400340F3400340034F70AA9
:1039A00008007708A200023C8A150A16031C0A2D9B
:1039B0008A150A160310220DA2078A150A16FA2480
:1039C0008A150A16A000A20A8A150A16FA248A1570
:1039D0000A16A100A20A8A150A16FA248A150A16DE
:1039E0008A110A12C4208A150A162008F1008A15C5
:0C39F0000A160A2D1D308A002208002D46
:103A000082070A34003400340234003400340F34A6
:103A100000340034F70A08007708A200023C8A1537
:103A20000A16031C422D8A150A160310220DA2073E
:103A30008A150A1635258A150A16A000A20A8A15C3
:103A40000A1635258A150A16A100A20A8A150A1631
:103A500035258A150A168A110A12C4208A150A16F3
:103A60002008F1008A150A16422D1D308A0022080E
:103A700082070A34003400347F34003400340F34B9
:103A800000340034F70A08007708A200023C8A15C7
:103A90000A16031C7A2D8A150A160310220DA20796
:103AA0008A150A166D258A150A16A000A20A8A151B
:103AB0000A166D258A150A16A100A20A8A150A1689
:103AC0006D258A150A168A110A12C4208A150A164B
:103AD0002008F1008A150A167A2D1D308A00220866
:103AE00082070A3400340034FF34003400340F34C9
:103AF00000340034F70A08000730BA004030B8003C
:103B00003C08AA003D08AB006430AC00AD018A114E
:103B10000A12DD208A150A168A110A12031C3E2B8E
:103B20008A150A16E2008A110A12DD208A150A1681
:103B30008A110A12031C3E2B8A150A16F1008514FD
:103B4000831685100F3083126205B200B3010E3068
:103B5000A000A1013308A30032088A110A121E2214
:103B60008A150A16ED006208A000A10104308A112E
:103B70000A1232228A150A16EE006308A100053CDB
:103B80008A150A16031CE62D8A150A16A10D8A1538
:103B90000A16D6258A150A16A00021108A150A16BB
:103BA000D6258A150A168A00200882001D308A0050
:103BB000210882071E3467341E346D341E3483346A
:103BC0001E3461341D34E6341E34F234ED016400D9
:103BD0000D306D028A150A1603185E2E8A150A1614
:103BE0008A114F208A1574088A110A125E208A15DC
:103BF0000A1666088A110A1263208A150A165430BA
:103C0000AA004030AB00AE01AF0108308A110A12A1
:103C100049218A150A1600308A110A1249218A158B
:103C20000A1674088A110A125E208A150A16543080
:103C3000AA004030AB003230AC00AD018A110A124C
:103C4000DD208A150A16031CF32DEF00E401640041
:103C5000033064028A150A1603185A2E8A150A16AA
:103C60006D086407B400B501B50D04306407B200F7
:103C7000B301B30D6F3084003208003E8A110A127E
:103C80004C208A150A160030031D0130B200B30122
:103C9000403084003408003E8A110A124C208A15F4
:103CA0000A16320C8A110A1257208A150A16E40ADB
:103CB000031D272E0330ED07031CE72D8A150A1676
:103CC000F82E0A1264270A168A150A16F82E0A1206
:103CD00018270A168A110A123E2B8A11BC208A154F
:103CE0000730BA008030B8003C08AA003D08AB009D
:103CF000AE01AF0171088A110A124F218A150A1606
:103D00008A110A123E2B8A114F208A1574088A11D3
:103D10000A125E208A150A1666088A110A126320A2
:103D20008A150A165430AA004030AB00AE01AF012C
:103D300008308A110A1249218A150A1600308A11A0
:103D40000A1249218A150A1674088A110A125E207D
:103D50008A150A165430AA004030AB003230AC004D
:103D6000AD018A110A12DD208A150A16031C862E5F
:103D7000EF006F3084006408003E8A110A124C2064
:103D80008A150A1603197110031D71146408A00026
:103D9000A10104308A110A122A228A150A16B200D9
:103DA0002108B3006F3084003208003E8A110A12E5
:103DB0004C208A150A160319F110031DF11407305F
:103DC000BA008030B8003C08AA003D08AB00AE0144
:103DD000AF0171088A110A124F218A150A168A1139
:103DE0000A123E2B8A11E8208A158A110A123E2BEC
:103DF0000730BA008030B8003C08AA003D08AB008C
:103E0000AE01AF0141088A110A124F218A150A1624
:103E100040088A110A124F218A150A168A110A12BD
:023E20003E2B37
:02400E00753DFE
:1042000000007F00FF007F00FF007F00FF007F00B5
:1042100000007F0000007F0000002800AA005A0074
:104220000400010002000300020005000200070074
:10423000FF000900FF000B00FF000F000100FF005E
:104240000500FF00090002000F000300FF00070047
:1042500002000B0002000F000300FF000900020033
:104260000F00000002000200FF0004000200060030
:1042700002000800FF000A0002000F000000FF001B
:10428000020002000400FF000600FF000800020018
:104290000A00FF000F0000007F0008007F000400FC
:1042A0007F000F0006007F0002007F000A007F00F1
:1042B0000F000000FF00020002000400FF000600E3
:1042C00002000800FF000A0002000F0000000200C8
:1042D0000200FF00040002000600FF0008000200C8
:1042E0000A00FF000F0000000000000001001100A4
:1042F000000011007300250052007500110011002C
:1043000073001E0075003E001100000011007300D4
:104310001E004B0075001100110073002500750090
:1043200031001100000011007300250052007500DB
:104330001100110073001E00750031001100000013
:10434000110073001E004B00750011001100730076
:10435000250075003E0011000000110073002500CB
:104360007500660011000000110073001E0075004A
:10437000590011000000110073001E007500660056
:104380001100000011007300250075005900110094
:1043900000001E004B00110025005200110000001B
:00000001FF
